:1000000003138316103085000F30860083120130F1
:100010009800FF3097008C01051E0B2800008C0F04
:100020000C288F011010051A13280F308C008C0B30
:100030001728051A00280515051108308D000F3006
:100040008C008C0B212805150511101D3A28151C54
:1000500030280512831600308500831200003728EF
:100060000516831610308500831200000000950CE1
:100070000A303B280E308C008C0B3C288E0C8E13E3
:10008000051E8E17051505118D0B1F280E308C00CF
:100090008C0B482805150511101D562805168316CA
:1000A00010308500831210110B3057280E308C0051
:1000B0008C0B5828051E0028051505118F0A0F0303
:1000C000073982076A2872287328742875287628C9
:1000D0007728782805150511901C712813089500BC
:1000E000101513281328132813281328132813284E
:1000F0008F01EE2090198820940B83280130940002
:1001000090101011872812089500901410150B28D4
:1001100096000F398207AA28A528A0289B28BE2868
:10012000B928B428AF28D228CD28C828C328E62863
:10013000E128DC28D728183092005E309300EB28A5
:100140002830920049309300EB2828309200473045
:100150009300EB282830920004309300EB282830DD
:10016000920077309300EB282830920051309300B2
:10017000EB282830920045309300EB28283092007D
:1001800014309300EB28183092009A309300EB283B
:10019000183092000B309300EB2828309200413049
:1001A0009300EB282830920061309300EB28183040
:1001B000920084309300EB28183092008630930030
:1001C000EB282830920053309300EB28183092002F
:1001D00033309300EB280430940008009011E03095
:1001E00086000000000006090F39031902290515D1
:1001F0000511960016183E2996184129161944290A
:1002000096194729D03086000000000006090F39F2
:100210000319152905150511960016184A2996186F
:100220004D291619502996195329B030860000001F
:10023000000006090F390319282905150511960034
:10024000161856299618592916195C2996195F29E6
:10025000703086000000000006090F3903193B29A1
:1002600005150511960016186229961865291619A4
:10027000682996196B291012FF306E29101600306C
:100280006E29101601306E29101602306E291012D8
:1002900003306E29101604306E29101605306E29B1
:1002A000101206306E29101207306E291012083015
:1002B0006E29101209306E2910160A306E29101698
:1002C0000B306E2910120C306E2910120D306E2971
:1002D00010120E306E2910160F306E29960017027C
:1002E00003197C29980B7F29033098001608970082
:1002F000FF3C031D90157F29101E7F2990151608BD
:020300000800F3
:00000001FF
